:1000000025C08BC63DC03CC03BC03AC039C038C0DB
:1000100037C036C035C034C033C032C031C030C044
:100020002FC02EC02DC0BCC8C0C8FBC8C0C8F9C8EE
:10003000C3C8C9C8CFC8D7C8F8C8F3C8F2C8F1C880
:10004000F0C8EFC8EEC8EDC8ECC8D4C811241FBE74
:10005000CFE5D4E0DEBFCDBF10E0A0E6B0E0EEED2E
:10006000FBE102C005900D92A438B107D9F711E069
:10007000A4E8B0E001C01D92A831B107E1F707C0C4
:10008000BFCF5D9BFECF8CB981E090E00895CBE4BB
:10009000D4E0DEBFCDBF14BA8FEF85BB17BA88BBE3
:1000A00011BA82BB88E08AB986E880BD89E189B946
:1000B00060E070E081E490E0C9D8909311018093F2
:1000C000100180E690E022D902D55BD678944DD716
:1000D000CE0101965DD58823D1F349815A819A01D9
:1000E00020702115310549F092E92030390709F4D3
:1000F00093C22050324159F7C0C34A3709F4CEC1E8
:100100004B3708F098C0413409F44FC2423408F02C
:1001100049C04B3109F453C24C31F8F44B3009F467
:100120000DC24C3050F4433009F4F9C34A3009F49D
:1001300044C1423009F086C49DC1423109F455C121
:10014000433120F4413109F07DC4B7C1433109F492
:1001500013C24A3109F076C464C14B3209F4D5C1E7
:100160004C3280F4423209F434C1433220F441323B
:1001700009F068C489C1433209F4EFC14A3209F079
:1001800061C407C1423309F43CC1433320F4413315
:1001900009F058C45EC1433309F4FDC1493309F085
:1001A00051C42BC24B3509F405C24C35F8F4413526
:1001B00009F47EC1423568F4433409F40FC2433474
:1001C00008F43BC14A3409F4E0C04B3409F03AC4A6
:1001D00097C1433509F4D5C1433508F40AC14935FF
:1001E00009F4DEC14A3509F02DC417C14B3609F4B4
:1001F000F0C14C3680F4423609F4EFC0433620F4A7
:10020000413609F01FC44FC1433609F4ABC14A3629
:1002100009F018C40EC1423709F413C1433720F462
:10022000413709F00FC419C1433709F4DCC149371C
:1002300009F008C4E7C1493B09F497C04A3B08F0FC
:1002400049C04A3909F4A9C04B39F8F44A3809F4CD
:1002500090C04B3850F4423809F4B3C0433809F425
:1002600072C1413809F0EEC300C1413909F42AC115
:10027000423920F44B3809F0E5C333C1423909F45F
:1002800094C0433909F0DEC34FC14A3A09F489C02A
:100290004B3A80F4413A09F4FCC0423A20F44B391D
:1002A00009F0D0C337C1423A09F46BC0433A09F0B0
:1002B000C9C321C1413B09F454C0423B20F44B3A2D
:1002C00009F0C0C32CC1423B09F4BFC0433B09F055
:1002D000B9C38EC1413E09F49CC0423E28F54B3C57
:1002E00009F436C14C3C80F4423C09F49EC0433CC6
:1002F00020F4413C09F0A6C3C2C0433C09F464C1E8
:100300004A3C09F09FC361C0423D09F476C0433DB9
:1003100020F4413D09F096C3DFC0433D09F436C1E6
:10032000493D09F08FC371C0413F09F49AC0423F73
:1003300060F4433E09F41BC1433E08F452C04A3EF8
:10034000E1F04B3E09F07EC3D1C0433F09F4F1C058
:10035000433F78F1493F09F45AC14A3F09F072C35B
:10036000B6C03EE41B8A1C8ADDC235E51B8A1C8AA6
:10037000D9C235E11B8A1C8AD5C23DE11B8A1C8A81
:10038000D1C234E21B8A1C8ACDC23DE21B8A1C8A80
:10039000C9C23CE21B8A1C8AC5C235E31B8A1C8A7F
:1003A000C1C23CE31B8A1C8ABDC233E41B8A1C8A7F
:1003B000B9C234E41B8A1C8AB5C23DE41B8A1C8A7C
:1003C000B1C23CE11B8A1C8AADC23BE11B8A1C8A7C
:1003D000A9C233E21B8A1C8AA5C23BE21B8A1C8A83
:1003E000A1C234E31B8A1C8A9DC233E31B8A1C8A88
:1003F00099C23BE31B8A1C8A95C232E41B8A1C8A81
:1004000091C23BE41B8A1C8A8DC23CE41B8A1C8A75
:1004100089C232E51B8A1C8A85C23AE11B8A1C8A82
:1004200081C232E21B8A1C8A7DC231E21B8A1C8A8D
:1004300079C23AE21B8A1C8A75C232E31B8A1C8A83
:1004400071C231E31B8A1C8A6DC23AE31B8A1C8A83
:1004500069C231E41B8A1C8A65C239E41B8A1C8A82
:1004600061C23AE41B8A1C8A5DC236E11B8AF1E054
:10047000FC8B58C23EE11B8A21E02C8B53C236E232
:100480001B8A81E08C8B4EC235E21B8A91E09C8BEB
:1004900049C23EE21B8AE1E0EC8B44C236E31B8A90
:1004A000F1E0FC8B3FC23DE31B8A21E02C8B3AC27A
:1004B0003EE31B8A81E08C8B35C236E41B8A91E0D7
:1004C0009C8B30C235E41B8AE1E0EC8B2BC23EE40E
:1004D0001B8AF1E0FC8B26C235E51B8A21E02C8BC0
:1004E00021C235E11B8A81E08C8B1CC23DE11B8A55
:1004F00091E09C8B17C234E21B8AE1E0EC8B12C2C4
:100500003DE21B8AF1E0FC8B0DC23CE21B8A21E03C
:100510002C8B08C235E31B8A81E08C8B03C23CE341
:100520001B8A91E09C8BFEC133E41B8AE1E0EC8BDB
:10053000F9C134E41B8AF1E0FC8BF4C13DE41B8A71
:1005400021E02C8BEFC13CE11B8A81E08C8BEAC15E
:100550003BE11B8A91E09C8BE5C133E21B8AE1E021
:10056000EC8BE0C13BE21B8AF1E0FC8BDBC134E3A6
:100570001B8A21E02C8BD6C133E31B8A81E08C8B54
:10058000D1C13BE31B8A91E09C8BCCC132E41B8A36
:10059000E1E0EC8BC7C13BE41B8AF1E0FC8BC2C1FC
:1005A0003CE41B8A21E02C8BBDC132E51B8A81E033
:1005B0008C8BB8C13AE11B8A91E09C8BB3C132E2CB
:1005C0001B8AE1E0EC8BAEC131E21B8AF1E0FC8BCF
:1005D000A9C13AE21B8A21E02C8BA4C132E31B8A19
:1005E00081E08C8B9FC131E31B8A91E09C8B9AC187
:1005F0003AE31B8AE1E0EC8B95C131E41B8AF1E020
:10060000FC8B90C139E41B8A21E02C8B8BC13AE42E
:100610001B8A81E08C8B86C1403809F4CEC04138FA
:1006200008F043C0403409F4CCC04134F8F44B31F5
:1006300009F4FBC04C3150F4403109F4DAC04831C0
:1006400009F4B3C0442309F4DCC0FCC1483209F406
:1006500092C0493220F4403209F0F4C1BAC04B32A2
:1006600009F4D3C0493309F0EDC1D3C0483509F4CA
:1006700064C0493550F44B3409F48BC0403509F45B
:1006800098C0423409F0DEC1CCC0403609F4A9C09C
:10069000413620F4493509F0D5C1DBC0483609F4AC
:1006A00060C04B3609F0CEC1CAC0403C09F48DC0D1
:1006B000413CF8F4483909F470C0493950F44938DC
:1006C00009F463C0403909F498C0483809F0BAC148
:1006D0003EC0403A09F481C0413A20F44B3909F058
:1006E000B1C1A8C0483A09F44BC0423B09F0AAC1C5
:1006F000B5C0403E09F479C0413E80F44B3C09F45A
:100700008CC04C3C20F4483C09F09CC125C0483DBD
:1007100009F4AEC0493D09F095C114C04B3E09F43F
:1007200093C04C3E20F4483E09F08CC11FC0423FAC
:10073000C1F1483F09F086C196C030E091E79B8B3C
:100740001C8AF0C030E0ECE6EB8B1C8AEBC030E09A
:10075000F4E2FB8B1C8AE6C030E022E22B8B1C8A81
:10076000E1C030E080E18B8B1C8ADCC030E099E195
:100770009B8B1C8AD7C030E0EEE2EB8B1C8AD2C088
:1007800030E0F0E3FB8B1C8ACDC036E71B8A1C8A65
:10079000C9C036E01B8A1C8AC5C034E01B8A1C8A8B
:1007A000C1C03CE01B8A1C8ABDC033E01B8A1C8A86
:1007B000B9C03AE01B8A1C8AB5C036E11B8A1C8A84
:1007C000B1C03EE11B8A1C8AADC036E21B8A1C8A7E
:1007D000A9C035E21B8A1C8AA5C03EE21B8A1C8A7E
:1007E000A1C036E31B8A1C8A9DC03DE31B8A1C8A7C
:1007F00099C03EE31B8A1C8A95C036E41B8A1C8A7A
:1008000091C035E41B8A1C8A8DC036E61B8A1C8A7F
:1008100089C03DE01B8A1C8A85C03AE51B8A1C8A78
:1008200081C039E21B8A1C8A7DC030E02BE62B8B0D
:100830001C8A78C030E084E78B8B1C8A73C030E060
:1008400092E79B8B1C8A6EC030E0E5E7EB8B1C8A3D
:1008500069C030E0FAE7FB8B1C8A64C030E02DE70A
:100860002B8B1C8A5FC030E08DE58B8B1C8A5AC0B5
:1008700030E090E79B8B1C8A55C0403519F141351B
:1008800068F4403161F1413118F4442361F1DAC078
:100890004034E9F0423409F0D5C00EC04039D9F0F7
:1008A000413920F4403609F0CDC030C0403A29F13A
:1008B000423C09F0C7C01BC030E0EDE7EB8BF1E034
:1008C000FC8B30C030E029E62B8B1C8A2BC035E036
:1008D0001B8A1C8A27C03BE01B8A1C8A23C033E882
:1008E0001B8A1C8A1FC031E01B8A1C8A1BC030E097
:1008F0008AE78B8B91E09C8B15C090E080918500FE
:10090000882309F491E090938500E1CB90E08091F9
:100910008400882309F491E090938400D8CB3EE0D2
:100920001B8A1C8A50918500552311F420E003C0D6
:1009300084E18B8321E040918400442331F0FE0167
:10094000E20FF11D81E183832F5F332381F1DE010B
:100950001396E22FFF27922F9F5F2C89222371F499
:10096000EA0FFB1F3083FD01E90FF11D80EF80834B
:10097000892F8F5FA80FB11D3C9339C0EA0FFB1F71
:1009800022E12083FD01E90FF11D3083892F8F5F64
:10099000FD01E80FF11D90EF90838F5FFD01E80FDF
:1009A000F11D30838F5FFD01E80FF11D1BC08B89A6
:1009B0008823F9F0DE011396FD01E20FF11D90EEA0
:1009C0009083822F8F5FFD01E80FF11D2B8920831B
:1009D0008F5FFD01E80FF11D90838F5FFD01E80F30
:1009E000F11D90EF90838F5FA80FB11D2C93282FDE
:1009F0002F5F442381F0FE013396DF01A20FB11D6A
:100A000080EF8C93922F9F5FE90FF11D81E180832E
:100A10002E5F10928400552381F0FE013396DF0192
:100A2000A20FB11D80EF8C93922F9F5FE90FF11DF4
:100A300084E180832E5F10928500822F992787FDA5
:100A4000909502C080E090E0F82E882309F43FCB17
:100A50008E010D5F1F4F0BC0F80180819DD101C039
:100A600084D294D18823E1F39CD10F5F1F4FCE0134
:100A70000396F02FF81BFF157CF329CB14BC8823B9
:100A800019F420E030E01CC020E030E00BC008B6D4
:100A900007FE05C088B7806888BF2F5F3F4F2617C5
:100AA00037078CF4829BF3CF10C008B607FE05C051
:100AB00088B7806888BF2F5F3F4F261737071CF421
:100AC0008299F3CF02C02FEF3FEFC90108958AE06A
:100AD00085BD88EC83BD14BC87E089BF82E085BFFB
:100AE00080E48BBF0895CF93DF93EC018A81282F98
:100AF00033278B81F901E80FF11DEF3FF10521F557
:100B0000E0918600F091870089819927982F8827A6
:100B1000822B932BEE0FFF1FE657FF4F91838083AD
:100B20008091860090918700019690938700809332
:100B3000860080918600909187008034910524F092
:100B40001092870010928600DF91CF910895E09176
:100B50008600F0918700EE0FFF1FE657FF4F8FEFE3
:100B60009FEF91838083809186009091870001960A
:100B700090938700809386008091860090918700F3
:100B80008034910524F01092870010928600089519
:100B9000DC014FB7F8942091860030918700809156
:100BA0008800909189002817390721F44FBF80E011
:100BB00090E00895E0918800F0918900EE0FFF1F0A
:100BC000E657FF4F808191818D939C934FBF809119
:100BD0008800909189000196909389008093880005
:100BE0008091880090918900803491051CF481E007
:100BF00090E00895109289001092880081E090E0C2
:100C00000895AF92BF92DF92EF92FF920F931F93DE
:100C1000CF93DF93CDB7DEB724970FB6F894DEBF3E
:100C20000FBECDBF5C018B0119821A821B821C8210
:100C300066E970E080E022DF8F5F9F4F09F45DC0BE
:100C400062E870E081E01ADF80559040459708F037
:100C500054C06CE370E080E011DF9C018FEF2F3F08
:100C6000380709F44AC0C9010A97459718F4F801F2
:100C7000099543C0295230402A30310508F03DC063
:100C8000E0E8DE2E00E010E0EE24FF2468E070E0F3
:100C900081E0F4DE0497049748F564E170E080E0B9
:100CA000EDDE9C018FEF2F3F380701F10032110577
:100CB00021F1C9010497059760F02E50304025308E
:100CC0003105D8F4FE013196EE0DFF1D80818D298E
:100CD0008083D69429F40894E11CF11C70E8D72E87
:100CE0000F5F1F4F0132110541F0D0CF00321105C7
:100CF00021F4CE010196F501099524960FB6F894DA
:100D0000DEBF0FBECDBFDF91CF911F910F91FF903E
:100D1000EF90DF90BF90AF9008951F920F920FB6A3
:100D20000F9211242F933F934F935F936F937F9371
:100D30008F939F93AF93BF93EF93FF9367EA75E011
:100D400083E795E05EDFFF91EF91BF91AF919F91B7
:100D50008F917F916F915F914F913F912F910F9064
:100D60000FBE0F901F901895A498AC9A8FEF9C9B84
:100D700003C080E090E008958150C9F781E090E0E1
:100D80000895A598AD9AA498AC9A0895809178009A
:100D9000992787FD9095089580930D011092780012
:100DA000089590E00BC0000000000000000000006B
:100DB0008F5F8634C1F79F5F983011F080E0F3CFEA
:100DC0000895FF920F931F93CF93DF93F82EA5986A
:100DD000AD9ACADF882309F0BCC09D9BBAC09C9B1A
:100DE000B8C0AD98A59A0000000000000000000007
:100DF0008F5F8634C1F7AC98A49A80E000000000B1
:100E00000000000000008F5F8634C1F7C0E0D0E032
:100E100011E001E0A9DF882309F09BC00000000079
:100E200000000000000000008F5F8431B9F78F2DB3
:100E3000812329F081E00827A598AD9A02C0AD98DA
:100E4000A59A80E0000000000000000000008F5F15
:100E50008634C1F79C9B7DC0AC98A49A80E00000CA
:100E600000000000000000008F5F8634C1F77CDFC7
:100E7000882309F06EC02196C830D10511F0110FFA
:100E8000C9CF72DF882309F064C0000000000000B1
:100E90000000000000008F5F8431B9F7002319F0D3
:100EA000A598AD9A02C0AD98A59A80E00000000018
:100EB0000000000000008F5F8634C1F79C9B49C092
:100EC000AC98A49A80E00000000000000000000040
:100ED0008F5F8634C1F748DF882309F03AC00000ED
:100EE000000000000000000000008F5F8431B9F7AF
:100EF000A598AD9A80E0000000000000000000000E
:100F00008F5F8634C1F7AC98A49A80E0000000009F
:100F10000000000000008F5F8634C1F7A498AC9AEF
:100F200080E0000000000000000000008F5F8634B9
:100F3000C1F78F2D99279F938F9388E690E09F9319
:100F40008F93D0D180E090E00F900F900F900F9092
:100F500006C0A598AD9AA498AC9A81E090E0DF9184
:100F6000CF911F910F91FF9008951F9380917B0067
:100F7000882319F08130B1F515C08091780088235D
:100F800099F580910A01882379F580910D0119DF87
:100F9000882351F581E08093780080910D01809342
:100FA0007A0022C08091790083301CF01092790081
:100FB0001BC08823C9F0813019F480917C0002C0E5
:100FC00080910B01FEDE882349F4809179008150E5
:100FD0008093790080910D0180937A00809179004F
:100FE000882311F410927B009C9B25C12DC19D99F3
:100FF00022C19D9902C09C9BFCCF9C9B1CC19D99CA
:101000001AC180E0000000000000000000008F5FB7
:101010008634C1F7AC98A49A80E00000000000007C
:10102000000000008F5F8634C1F7A498AC9A80E07E
:10103000000000000000000000008F5F8634C1F750
:1010400041E010E091E020E030E051E0AC98A49A5B
:101050009D9B02C04527192B80E000000000000086
:10106000000000008F5F8634C1F7A498AC9A80E03E
:10107000000000000000000000008F5F8634C1F710
:101080002F5F3F4F2830310511F0990FDFCFAC981B
:10109000A49A23B380E000000000000000000000DC
:1010A0008F5F8634C1F7A498AC9A80E000000000FE
:1010B0000000000000008F5F8634C1F7AC98A49A4E
:1010C00093B380E0000000000000000000008F5F8C
:1010D0008634C1F7A498AC9AAD98A59A80E0000038
:1010E00000000000000000008F5F8634C1F7AC985C
:1010F000A49A80E0000000000000000000008F5F64
:101100008634C1F7A498AC9AA598AD9A95FF19C0FA
:10111000822F8072442319F0882399F002C088231B
:1011200081F4812F99279F938F9380E790E09F937D
:101130008F93D8D00F900F900F900F901E3F81F497
:1011400007C08EEF80937C0081E08093790079C0A6
:1011500081E08093790080917A0080937C006BC05D
:1011600080910C01813009F45EC082301CF4882328
:1011700041F061C0823009F446C0833009F05BC0A1
:1011800052C00FDE812F9927AA27BB27FC01ED5EF5
:10119000F040E331F10508F044C0ED5EFF4F0994E3
:1011A0008AEF80937C0081E012C08EEE3FC08AEF10
:1011B00080937C0082E00BC083E880937C008BEA04
:1011C00080930B0129C08AEF80937C0083E0809399
:1011D0000C012EC08AEF80937C0083E080930C0189
:1011E00010920A0125C08AEF80937C0081E08093F1
:1011F0000A011EC010920A018AEF80930B018AEA4D
:1012000080937C0009C0112351F480937C008AEF05
:1012100080930B0110920C0182E090E00FC012301D
:1012200021F08EEF03C010920C018AEF80937C00B6
:1012300081E090E003C09C9BDACE06C080937900E9
:1012400081E080937B00F7CF1F910895EF92FF928A
:101250000F931F93CF93DF938C017B01892B11F4A4
:10126000672BC9F16EE070E081E090E0F9D2FC01FB
:10127000009789F1DC0180E88383E114F10471F0C7
:10128000F386E28681E8838380910E0190910F01BD
:10129000892B21F4F0930F01E0930E010115110544
:1012A000E1F0118700878381826083838091100140
:1012B00090911101892B89F4F0931101E0931001B1
:1012C0008091120190911301892B39F4F09313014D
:1012D000E093120102C0A0E0B0E0CD01E6E0CDB79E
:1012E000DEB76EC4A2E0B0E0E7E7F9E051C4FE016A
:1012F000379661917191FA83E983AF018091100172
:101300009091110136D0E2E022965EC40F931F93B4
:10131000CF93DF938C01E0911001F0911101838153
:1013200081FF1FC0C0E0D0E00AC0FD0120853185EB
:10133000BD01F9010995892B11F0CFEFDFEFF8011D
:1013400081918F01A0911001B0911101882369F75B
:10135000FD0120853185BD018AE0F9010995892BC0
:1013600011F0CFEFDFEFCE01DF91CF911F910F9101
:101370000895A2E1B0E0EEEBF9E0FAC388249924E5
:1013800054012C017A8B698B3A01FC011782168279
:10139000838181FD03C08FEF9FEF5FC2CC24DD24EA
:1013A0004BC2C0FE33C2832D80538A30E0F4F0E399
:1013B0003F1641F42D85222329F4C3FC03C080E0AD
:1013C00091E078C08AE0ED85E802C0011124380E72
:1013D000F32DF053FD87F7FF02C02FE72D87C3FCE5
:1013E00026C22D8424C2C60188709070C3FE05C039
:1013F0003D85332311F4E1E0ED87F7E6F3156CF159
:1014000025E632160CF067C033E5331609F486C0C2
:101410003315BCF08BE2381609F441C083154CF04B
:1014200090E2391609F43FC0E3E23E1609F0E5C147
:1014300044C0FDE23F16E1F12EE2321609F0DDC1B3
:1014400041C033E6331609F44CC033150CF47DC0AB
:1014500088E5381609F0D1C11FC0E0E73E1609F44F
:101460009EC0E3155CF0FCE63F1691F12FE63216C4
:1014700089F039E6331609F0C0C167C0E5E73E16CA
:1014800009F495C0F8E73F1639F023E7321609F062
:10149000B4C12FC038E08AC080E1888B88C0E0E109
:1014A000F0E0CE2ADF2A20E230E0C22AD32ABFC1F0
:1014B00080E890E0C82AD92ABAC1E0E4F0E0CE2A58
:1014C000DF2AB5C128E030E0C22AD32A1D86AFC189
:1014D00084E090E0EFCF5FE3852E2A9443E6342E3C
:1014E00028C1F30180802A9422E030E0620E731E4E
:1014F00020C1F30180809180892B41F0FD856F2F01
:10150000772767FD7095C401D9D217C0F401019007
:101510000020E9F73197E819E88B10C0F3018080CB
:101520009180892B41F0FD856F2F772767FD70959E
:10153000C401B2D202C0C401A6D2888B22E030E03E
:10154000620E731E3889231AF4C0C2FE08C0F3016C
:1015500080819181A281B38124E030E009C0F30150
:1015600080819181AA2797FDA095BA2F22E030E0D3
:10157000620E731E4C015D01B7FF0CC082E090E06B
:10158000C82AD92AB094A09490948094811C911C6C
:10159000A11CB11CEFEBFFEFCE22DF2221C020E423
:1015A00030E0C22AD32A38E7332E30E1388BC2FE2E
:1015B00008C0F30180819181A281B38124E030E0F1
:1015C00007C0F30180819181AA27BB2722E030E088
:1015D000620E731E4C015D018FEC9FEFC822D92271
:1015E00085017401FE013196FF87EE87F8898F2E01
:1015F0009924AA24BB24C801B701A501940196D25D
:101600006A301CF0630D615201C0605DEE85FF859C
:101610006193FF87EE87C801B701A501940186D2C7
:1016200079018A01211531054105510521F78824E9
:1016300099245401CE0101968E84881AC6018273C2
:101640009070892B09F02A94C6FE07C0F889F03102
:1016500011F482E001C081E0281A28E0E22EF12C8A
:10166000EC20FD20C3FE16C08D85282F332727FDD3
:101670003095882D9927821793073CF0E7EFFFEF0D
:10168000CE22DF22EE24FF2405C0FD85F819FD8758
:101690002F1A01C02818C60180789170892B61F437
:1016A000822D05C0B20180E290E013D2812F182F65
:1016B00011501816BCF3212EC1FE04C0B2018DE2F8
:1016C00090E00BC0C4FE04C0B2018BE290E005C004
:1016D000C5FE04C0B20180E290E0FBD1C6FE0DC0A1
:1016E000B20180E390E0F5D12889203131F4B201D4
:1016F000832D992787FD9095ECD1D0FE0CC0822DCB
:1017000005C0B20180E390E0E4D1812F182F115081
:101710001816BCF3212EEF2861F02D8505C0B2010B
:1017200080E390E0D6D1212F122F11501216BCF376
:101730001D8790E8E92EF12CEC20FD20C7FC0CC0A1
:10174000822D05C0B20180E290E0C3D1812F182F15
:1017500011501816BCF3212E33E6331639F4B201BA
:10176000882D992787FD9095B4D138C083E7381626
:1017700081F4840108C0F80181918F01B201992799
:1017800087FD9095A6D1F889F150F88BFF3F99F726
:1017900014C023E5321619F00E851F8518C0840188
:1017A00007C0F8018491B201992793D10F5F1F4FB1
:1017B000F889F150F88BFF3FA1F748010FC0F801FD
:1017C00082918F01B201992787FD909582D1CE0138
:1017D00001960817190799F71F870E87EF2899F0C8
:1017E000822D05C0B20180E290E073D1812F182FC5
:1017F00011501816BCF3212E06C0B201832D992773
:1018000087FD909566D1CC24DD2411C0F5E23F160A
:1018100041F42AE0288B22241D8681E0C82ED12C99
:1018200006C0B201832D992787FD909552D18989F1
:101830009A8901969A8B898BF201838183FF04C078
:10184000E989FA89349003C0E989FA893080332024
:1018500009F0A7CDF20186819781E2E16296A4C1E9
:101860000F931F93CF93DF93869F8001879F100D67
:10187000969F100D1124C8010DD0EC01009721F0A6
:10188000A80160E070E013D1CE01DF91CF911F91EC
:101890000F910895CF93DF93AC01029710F442E0CB
:1018A00050E0A0911601B0911701FD01C0E0D0E019
:1018B00020E030E020C0808191818417950769F491
:1018C00082819381209719F09B838A8304C090932F
:1018D000170180931601CF0132C04817590738F419
:1018E0002115310519F08217930708F49C01EF01C7
:1018F0000280F381E02D3097F1F62115310589F151
:10190000C901841B950B049708F4A901E0E0F0E0FD
:1019100026C08D919C91119782179307E9F448177F
:10192000590779F4ED018A819B81309719F09383EF
:10193000828304C09093170180931601CD01029613
:1019400049C0841B950BFD01E80FF91F419351938A
:1019500002978D939C933AC0FD01A281B3811097A9
:10196000C1F68091140190911501892B41F4809169
:101970007F00909180009093150180931401209135
:101980008100309182002115310541F42DB73EB719
:1019900080917D0090917E00281B390BE09114010D
:1019A000F09115012E1B3F0B2417350788F0CA0153
:1019B00002962817390760F0CF01840F951F029611
:1019C000909315018093140141935193CF0102C06C
:1019D00080E090E0DF91CF910895CF93DF9300975F
:1019E00009F44EC0EC0122971B821A82A0911601C5
:1019F000B0911701109711F140E050E001C0DC01F7
:101A0000AC17BD0700F1BB83AA83FE012191319180
:101A1000E20FF31FEA17FB0771F42E5F3F4F8D9122
:101A20009C911197820F931F99838883FD01828176
:101A300093819B838A834115510559F4D0931701F3
:101A4000C09316011DC0FD0182819381AD010097F5
:101A5000B1F6FA01D383C28321913191E20FF31FD2
:101A6000EC17FD0769F42E5F3F4F88819981820F43
:101A7000931FFA01918380838A819B819383828360
:101A8000DF91CF910895FC0105900020E9F7809542
:101A900090958E0F9F1F0895FC0105906150704036
:101AA0000110D8F7809590958E0F9F1F0895DC0147
:101AB00001C06D9341505040E0F70895FC01615022
:101AC000704001900110D8F7809590958E0F9F1F60
:101AD00008950F931F93CF93DF938C01EB018B81BC
:101AE000992781FF1BC082FF0DC02E813F818C8111
:101AF0009D812817390764F4E881F9810193F983FE
:101B0000E88306C0E885F985802F0995892B31F493
:101B10008E819F8101969F838E8302C00FEF1FEFFE
:101B2000C801DF91CF911F910F910895A1E21A2E64
:101B3000AA1BBB1BFD010DC0AA1FBB1FEE1FFF1F71
:101B4000A217B307E407F50720F0A21BB30BE40BC1
:101B5000F50B661F771F881F991F1A9469F7609508
:101B60007095809590959B01AC01BD01CF010895C2
:101B70002F923F924F925F926F927F928F929F929D
:101B8000AF92BF92CF92DF92EF92FF920F931F938B
:101B9000CF93DF93CDB7DEB7CA1BDB0B0FB6F8943C
:101BA000DEBF0FBECDBF09942A88398848885F847C
:101BB0006E847D848C849B84AA84B984C884DF80ED
:101BC000EE80FD800C811B81AA81B981CE0FD11DD1
:0E1BD0000FB6F894DEBF0FBECDBFED01089535
:101BDE006972327073320D003C253032780D0A0076
:101BEE003E253032780D0A000101FF01AA200018AF
:041BFE0001000000E2
:00000001FF
